:103E0000112484B714BE81FFE7D085E08093810040
:103E100082E08093C00088E18093C10086E08093B7
:103E2000C20080E18093C4008EE0C0D0259A86E075
:103E300020E33CEF91E0309385002093840096BB13
:103E4000B09BFECF1D9AA8958150A9F79924939411
:103E5000A5E0AA2EF1E1BF2E9DD0813421F481E0AE
:103E6000B3D083E01FC0823411F484E103C08534F1
:103E700019F485E0A9D083C0853579F48BD0E82E7C
:103E8000FF2488D0082F10E0102F00270E291F29AB
:103E9000000F111F91D0680172C0863529F484E0AB
:103EA00093D080E06FD06BC0843609F042C072D0EE
:103EB00071D0082F6FD080E0C81688E3D80620F4B0
:103EC00083E0F60187BFE895C0E0D1E063D0899335
:103ED0000C17E1F7F0E0CF16F8E3DF0620F083E0FF
:103EE000F60187BFE89568D007B600FCFDCFA601B4
:103EF000A0E0B1E02C9130E011968C91119790E008
:103F0000982F8827822B932B1296FA010C0197BECB
:103F1000E89511244E5F5F4FF1E0A038BF0751F7DD
:103F2000F601A7BEE89507B600FCFDCFB7BEE89541
:103F300026C08437B1F42ED02DD0F82E2BD03CD013
:103F4000F601EF2C8F010F5F1F4F84911BD0EA9475
:103F5000F801C1F70894C11CD11CFA94CF0CD11CF4
:103F60000EC0853739F428D08EE10CD084E90AD010
:103F700086E098CF813511F488E018D01DD080E11B
:103F800001D06ACF982F8091C00085FFFCCF90931D
:103F9000C60008958091C00087FFFCCF8091C000CB
:103FA00084FD01C0A8958091C6000895E0E6F0E088
:103FB00098E1908380830895EDDF803219F088E0E6
:103FC000F5DFFFCF84E1DECF1F93182FE3DF115021
:103FD000E9F7F2DF1F91089580E0E8DFEE27FF2781
:023FE000099442
:023FFE000304BA
:0400000300003E00BB
:00000001FF
